:020000040000FA
:10000000850186018316EC2AFF00FF0E030E830193
:10001000D3000408D4008C10BE0B11283230BE006F
:10002000BD17C7082B1C0319172886161828861217
:10003000AA0F2A28A90F2A28AB0A7D153C30AA004E
:10004000F630A9002B182A28C708031DC70B2A2839
:1000500006128612CB186F28CB1D3428CC0B6F28C4
:100060000519CB11CC0A6F284B1C3E2805196F28A7
:100070004B10CD010430CE0006305F2805084B063A
:10008000043903194928CB064B1602304B1B0630A6
:10009000CC004B1B5628CC0B6F28031005190314FA
:1000A000CE0DCD0D4B174B1204305F284B1A612833
:1000B000CC0B6F284B0882390938CB008030CC003C
:1000C0006F284B13CD1F6F28CE0DCD0D4E0DCD0DCE
:1000D000CE134D1FCE17CD1A0314CE0CCB14851E94
:1000E000C303851AC30AC20BEF286430C200C00ADA
:1000F0000319ED280301C31B2030C301C3174106B8
:1001000020390319EF28C106411C9628C11A9D28E1
:10011000B5304007031C8F28E73E031C912841118E
:10012000EF28E430C105BF01BF039828C11A9F28FA
:10013000E2304007031CED28BF0AC001EF28F13070
:1001400040070318ED28F9304007031CA928C11700
:10015000AE28FD304007031CED28C113C00141113A
:10016000C63084003A303F020319DF28083E0318E6
:10017000D92880018403083E0318D928800184030C
:10018000063E0318D92880018403013E0318DF28A6
:10019000063E0318D92880018403013E0318DF2896
:1001A000073E0318D9288001013E0318C11BEF2820
:1001B000ED28410D800C0830C11BC106EF28083026
:1001C000C11BC106C119EC283A303F060319C118FA
:1001D000EF28C40A4115EE284116C11441145408F1
:1001E0008400530E83007F0E0900AB013C30AA004F
:1001F000F630A9000800F101F10AF63E0318FC28C8
:100200000A3EF103F10E7107080060261C21031D50
:100210000D294808C70006161721F10B06291C21D5
:10022000031D080063080319013EE2005715A824C6
:100230007D141E25FD1408002D080006F000840A18
:100240002C080006840A70040800FD101F3071217C
:10025000FD1B2B1C482186102530840007308A00A6
:1002600000081F39CA27801B40387D1C0030FB0066
:1002700008300611FB1F8611FB1B8615FB0D0615AA
:10028000FF3E031D39298403841A2E298614080091
:100290002B1C4C29571970297C1A1C2A8A007C08AF
:1002A0000F398207002AF329EA29C7299C29AE2998
:1002B000B62986297D297829182AC129D729D7293D
:1002C000D72951080F39A100510E0139A00018306B
:1002D000A2001E30A30052080F39A500520E152AA5
:1002E0000830A000A100A200A300A400A5000134D2
:1002F0001830A200A3006108CF2957080339E5216F
:100300000A30A2001A30A3005508CF29FE1B9329FA
:100310007E0828073F39E5210030A71B323E271B06
:10032000193EED2197291B30A000A100A200A117C2
:100330001D30A4000C3076290D30A0000C307D1F3C
:100340001E30A1004508CF214408D321A300A921D4
:10035000F129700E0F3903191F3008004908E521F3
:100360001130A2000530A3004A08CF291A303D18E9
:100370000D30A0000530A2000E30A3007D0E033921
:10038000CF291830A2000D30A3006308CF290D300B
:10039000A2000A30A300330AE521FD190C30D32155
:1003A000A500A921162AFB20F0000F3908004C3EB9
:1003B0008400000E0F39CF210B30A200041C103036
:1003C00084181830A300570E0739D321A100A921A2
:1003D000A00018343108FA213008D321A300700E90
:1003E0000F39A20008002F08ED212E081222300834
:1003F000FA210F2AD321A100700E0F39A0000800A6
:100400002D08FD19B324E5212C08ED212F221222FD
:100410002B1C080044084507E23E0318A517A11746
:10042000A3170800D321A500700E0F39A4000800FF
:10043000C030840018301F2AA2247C080F39A10084
:100440000A30A0001830000603192C2A0008A52144
:10045000A317840A0008122AA3010F30752903107C
:100460002B0C08009B25CB174D08D10050061F39D7
:10047000D01B0039031DE52A4E08D200CF06031910
:10048000E52A7F39F0004030F100F11AE52A7108C1
:100490004827F10A7006031D452AFD1402308A0020
:1004A00071031F398207832A7E2A862A8B2A952A7E
:1004B0009C2AA42AAD2AB52ABE2AC62ADF2ACE2A19
:1004C000DD2ADA2A732A772A752A4F2C742C0A2DF2
:1004D0000A2D0A2D0A2D0A2D0A2D4C2DF02CCF2C79
:1004E000C62CCD2CC82CC701E52A4625E52A792241
:1004F000E52A7C0A7C061F39FC061A29AB0AAB0ADE
:1005000078302B020318AB01F620E32AAB027830D7
:10051000031CAB07842A8D22E32AAC0A3C302C064C
:100520000319AC0008003D1C8D2A9722E32AAC0376
:10053000AC1FE32A3B30912A9E22E32AAD0A1830F1
:100540002D060319AD000800A822E32A3D1C9E2AAF
:10055000AD03AD1F08001730A22AAF22E32A3203F1
:100560002E060319AE01AE0A0800B922E32A3D1C8B
:10057000AF2AAE0B08003203AE000800C022E32A07
:100580000C302F060319AF00AF0A0800CA22E32A75
:100590003D1CC02AAF0B08000B30C32AD022E32A2F
:1005A000B0036330B01F0800B000B1036330B11B6B
:1005B000B1000800D5220230E12AB10ADB2AB00AD4
:1005C0000130FC00E42AFC0101264E08CF00CB10CC
:1005D000CB1F0800ED241729C03086008112F930A6
:1005E00092008C14831207309F0020308400800119
:1005F000840A841FF72AC603C3176430C20041145B
:100600003E3048273F390319013EC8003F30482794
:10061000D0004B14603048270739483EE400E40717
:100620006408F8000130F90020300A275425EB2631
:100630000A275925EB260A2743250130F526A0383D
:10064000E500A8250D261721053092008C01C03049
:100650008B00CB18322241081739043A0319DA25E6
:100660007D1D762BFD14A3264E27B300640AF800E7
:10067000F901F626A70043252B18432BA608031DD6
:10068000A60B432BFC017125FC08031D502B2B06E8
:100690007D1B031D502BED2401302C1C0730FC006A
:1006A000AB08031D762BD608031DD60B592B571804
:1006B0004825E20857190319602BE20B602B5711EC
:1006C00046082C060319662BC60605212C08031DB7
:1006D000762B4408C500C4019924C7080318031DDC
:1006E000762B0130FD1AB3247D1AC7002C03FB00C2
:1006F0001E302B067B04031D882BAF242D08F3002E
:1007000061080319882BF500A4277608031D052628
:10071000FD182521BD1F2F2CBD130310051E03142A
:10072000B40D34090319A02BC03A32300319B800B4
:100730003408FE3A031DA72B3C1EA42B3C12A72B0A
:10074000B80BA72B3C16FC173C143230B800031032
:10075000851D0314B50D35090319BA2BC03A323083
:100760000319B9003508FE3A031DC12BBC1EBE2B70
:10077000BC12C12BB90BC12BBC16FC17BC143230F8
:10078000B9003C0830390319FC133C1CF82B3C1011
:10079000EA243C1ACD2B46252F2C7D1CCB2BA824DC
:1007A000A2247C1A2C2C0330AB248207A6222E2CE8
:1007B000C8222E2C6D252E2CFD11322C7D13322CAF
:1007C000C90AFE2C1030302CA80ABC2CDD242F2C9A
:1007D000F2242F2CF5232F2C5B252F2C4F252F2C8B
:1007E0004F252F2C4F252F2C2F2CC03084002C2C44
:1007F000BC1C2F2CBC10EA24BC1A042C7D1C022C1F
:1008000079222F2C46252F2C7D1C022CA824A024D5
:100810007C1A2C2C0430AB24820793222E2CB72276
:100820002E2C69252E2CFD15322C7D17322CCA0A50
:10083000FE2C07252F2CA803BC2CDB242F2CF42402
:100840002F2C3D242F2C65252F2C0F252F2C0F25E9
:100850002F2C0F252F2C2F2C3F242F2C0126292B1A
:1008600034242F2C38242F2C7D077D063039FD06AB
:100870001430F9007D0878390A2FC1308400800ACD
:10088000041004087F39F900193047243C30801BDC
:1008900080070002031880000008840A0A2FA2249F
:1008A0007C1AD22C0430AB248207A622C22CC82288
:1008B000C22C6D25C22CFD11D52C7D13D52CC90A57
:1008C000D72C1030D92CA80ABA2CDD24E52AF22422
:1008D000E52AF523E52A5B25E52A4F25E52A4F255C
:1008E000E52A4F25E52AE52AA0247C1AD22C0430DB
:1008F000AB2482079322C22CB722C22C6925C22CBA
:10090000FD15D52C7D17D52CCA0AD72C0725E52A2D
:10091000A803BA2CDB24E52AF424E52A3D24E52AA1
:100920006525E52A0F25E52A0F25E52A0F25E52A65
:10093000E52A49082D02031C08002D0A4A02080076
:100940000314A32C03107C0D1F39A03E8400080063
:100950005508D60008008A007C0D1E390800F001F9
:10096000F101F20108002D08F43E031C2D080319C3
:100970000C3E0800BE24E52ABE242F2C1730F900B7
:1009800028080A2FFD137D15CB16E52AA224C92CB1
:10099000A0247C1EE52A8003D32CA024D02CA224E2
:1009A0007C1EE52A800A4024E52A3824E52A002511
:1009B000E52A3424E52AD50AE22C013057075706E8
:1009C0000339D7061930F90057080A275530840033
:1009D0006430472CA824C701FD140A30A600080083
:1009E0001030E12AE103F52CE10A1930F90057082B
:1009F0000A271B30F90061308400052D00252F2CBB
:100A00001530F9004930840005251830472C013095
:100A1000BD0608009C3E10250408B43EE12A993E1C
:100A20008400840C1030031CF03080071D30F90066
:100A300058080A2759080A275A080A275A08F400AA
:100A4000590E58047D18382DF4012F22FB20F10E89
:100A5000F10A0F390030D718031D382D1030571FF9
:100A6000382D7119F4041130F11CF039711C0F3953
:100A7000F300522573080A27740E0A2757257308B6
:100A80000A27740E0A27A030F8003C347D1C172971
:100A9000D6017D10CB131E2D4F250C30E12A1030CE
:100AA000D707F52C1430F9004030F800003414302A
:100AB000F9004230552D63083B3A031D3B3A013E95
:100AC000E3001C30F90063080A2F630B682D3B30EC
:100AD000602D3D18D02AB00F08003D18D52AB10A64
:100AE0000800571E1E2D2F2203390319571E882D6B
:100AF000D71A812D9625DE079625DF079625E00774
:100B0000882DB025DE00700EF039DF008D25E00065
:100B1000600EF4005F0E5E04222D0F30F00570159C
:100B2000B025F00B902DF000F03908009D25650EE2
:100B30006506103908000108E5060310E50D650E8D
:100B4000E039E50C650765076507353CE5000800F9
:100B50009D25E600650EE7009D25E900650EE8008D
:100B60006608EB00EC00EA006708ED00EE00ED0D12
:100B7000EB0DED0D6B0DEA06EC0CEE0C6E08EA06C3
:100B8000EC0C6E0CEA066708E6006808E7006908E6
:100B9000E8006A08E90008008403000CF000700C0B
:100BA0003F39F3000F39731A0A3EF31A143E731BD0
:100BB000283E0800C63084000008D1253006F10028
:100BC000B0068403000CF000F00C700C1F39D12526
:100BD0002F06F104AF06CC252E06F104AE06CC2577
:100BE0002D06F104AD068403000C7F39D1252C06B7
:100BF000F104AC062F22F1044111F520F10803198C
:100C000008007D15CB16FD1308001030F526F60000
:100C1000F626FF3A7606031D0800F5200130F5267A
:100C2000B03EAB0DF626D125AB07AB07F626D12596
:100C3000AC00F626D025AD00F626D025AE00FA0E83
:100C4000FA0C7A0CF200F6261F39D125AF001030CD
:100C5000F526B000F626FF3A3006031D672E123047
:100C6000F526B100F626F6267D067839FD06F6262D
:100C7000C900F626CA00F626A800F626F62657066C
:100C8000FB39D706F626D500F626E100F626E30066
:100C9000F626D800F626D900F626DA006026F10AF4
:100CA000F6268000840AF6268000840AF10B502E76
:100CB00030087206033903190800B00AA326E32E90
:100CC0002030F900A03084001030F10008000C3012
:100CD000AD00AC01AB010130AE00B301AF00B0001C
:100CE0001430B1001330F9000030FC000A27FD1762
:100CF0000A270830C9000A271430CA000A27003022
:100D0000A8000A270A270330D7000A275A30D5003F
:100D10000A270630E1000A271E30E3000A27703058
:100D2000D8000A27D9000A27DA000A276026F10A24
:100D3000183080000A27840A003080000A27840ABD
:100D4000F10B982E08002B3084007830EE263C30D2
:100D5000EE261830EE262030B2002F08F000AF1932
:100D6000F00A701CB203023A031DBD2EB203300814
:100D7000031931080339031DB2033208EE260318A4
:100D8000AE0A0D30EE260318AF0AEE263102031824
:100D9000B1017D11CB1E08008030EC2603012B1819
:100DA000503E09272F2209272C0809272D0809273B
:100DB0002E08FB2030184038B01880380A272F083A
:100DC0000927EB26CB121030F90030080A2730092A
:100DD0000A2731080A2F0030F9010A2F00020318F0
:100DE0008000840A0318800A6434F9001527282734
:100DF0002727152701382827781C022F1A277A0859
:100E0000FE0033271A2735271127F90A7A0883129B
:100E10000800FB20FA001527282727277A0828270B
:100E2000042F372740278514412F83161327402787
:100E300037273E2F1327F3154027831203108518F9
:100E400003148316FA0D3E27F30B1C2F08007908B4
:100E5000FB000830F300FB1B1327FB1F3727392744
:100E6000FB0DF30B2B2F3727362F13273927851030
:100E7000412F05140830FF3E031D3B2F0510412F65
:100E800005140830FF3E031D422F7808FE39080084
:100E900083169B001C141A0883010800AF242E0837
:100EA000F3003008F600F7013108F40003195E2F53
:100EB0006430F6070318F70AF40B582F2F08FD3E8D
:100EC000F400F41F662F0C30F4078317C227730752
:100ED000F200831F6F2FF603760A0319F703770CCE
:100EE000F400760CF3006D30F2070130C727F107EC
:100EF0000318F00AF60B732FF703F71F732F1F3039
:100F0000F2074330C727F1071A30C727F007F40C60
:100F1000F30C3108831F8F2FB0080319FF3EF60032
:100F2000F302031CF403F60C760C3F397307031825
:100F3000F40AF2077408C727F1070318F00A8301BF
:100F4000F501F3010730FB00F601F7012030F40052
:100F5000F30DF20DF10DF00DF60DF70DF40D750812
:100F6000F6027B08031C7B0A7702031874147418BA
:100F7000BC2F7508F6077708F7000310F40CF40B84
:100F8000A82F080007308A007408F23E8200031878
:100F9000013E08008207B734A0343B34B934AC3486
:100FA0009D349F34B034BF34BD34BE348F341734D5
:100FB000AB341F341E349734AE340634A1340734B6
:100FC0008A348B343E340A340F34A734083409345D
:060FD0003C340B34003438
:0C0FE40000341F343D345C347A349934FE
:100FF000B834D634F534E23EE23E543EF10A0800FD
:084000000700020004000800A3
:02400E00423F2F
:10420000360020007400750062006500200049003F
:104210004E002D00360020005600460044002000CD
:1042200063006C006F0063006B0020007700690082
:104230007400680020004400430046003700370047
:104240002000730079006E006300680072006F0048
:104250006E002C0020004900320043002000520074
:10426000540043002C002000520047004200200070
:0A4270004C006500640073002E008E
:04427C000800100026
:1042800010001C001800150011001D001900160078
:1042900012001E001A00130017001F001B00000070
:1042A0000F00030009000500300031003400350024
:1042B000320033003F000E000B000A00070006002A
:1042C000030048007000340031004300200020004B
:1042D000560032002E00340038002000320030003A
:1042E000310032002D00300035002D003100320049
:1042F00020005000430046003800350038003300ED
:00000001FF
